:1000000009C016C015C0C1C013C012C011C010C0B5
:100010000FC00EC011241FBECFE9CDBF20E0A0E667
:10002000B0E001C01D92A137B207E1F7EDD051C198
:10003000E7CFC09AC198089581E087B983E886B96F
:10004000369A3699FECF84B195B123E0969587957F
:100050002A95E1F78158089583E087B983E886B946
:10006000369A3699FECF84B195B196958795969537
:1000700087950895CF93DF93D82FC92FEDDF682F91
:100080008D2F9C2FDF91CF9117C10FC18111D1CF3F
:10009000C19AC098089588B38C7F88BB08950F9348
:1000A0001F93CF93DF93D82FC7DFD6DFC82F8D17CD
:1000B00050F48D2F8C1BC82FC11107C0DF91CF9139
:1000C0001F910F910895CD1BF7CFC6DF082F8D1715
:1000D000B0F4CD2FC81B1FE7C13220F0ADDF182FC1
:1000E0000D1790F4A6DF80E0811311C0D4DF1F3F0D
:1000F00019F382E08A95F1F700C01F5FF8CFC82F8F
:10010000CD1B1FE7C13250F780E0C0DFECCF92E09B
:100110009A95F1F700C08F5FE7CF8FEF80936D0066
:1001200080916E00807F80936E0010926F0084E05B
:1001300080937000BC98C49A8BED95E00197F1F71D
:1001400000C00000E199FECF90E080E0AED08A3A96
:1001500099F481E090E0A9D0A2DF109261001092A2
:1001600060001FBC13BE83B7836083BF789412BE48
:1001700089B7826089BF08956AEA90E080E09CD0E8
:100180006FE781E090E098D0E8CF1F921FB61F92F2
:1001900011242F933F938F939F93EF93FF93F894A2
:1001A000E0916200F0E086B3ED59FF4F80838091CB
:1001B00062008F5F8093620090E080E02FEFFC018F
:1001C000ED59FF4F3081232301968A309105B9F70D
:1001D00020936D00809162008A3010F010926200CE
:1001E00080916E0083FF05C080916F008F5F8093C8
:1001F0006F007894FF91EF919F918F913F912F9194
:100200001F901FBE1F90189588DF80916E0080FFA1
:1002100029C0846080936E00982F9A7039F4857F8E
:10022000886080936E0010926F000AC083FF08C040
:1002300090916F00923420F0857F826080936E00F1
:1002400080916D0090E02091700002C09595879597
:100250002A95E2F790916E009E7F80FF91609093C7
:100260006E00D3CF81FF07C081E090E003DF809173
:100270006E00817FD6CF82FF16C0EEDEC82F81E0F0
:1002800090E013D0C81748F48C1BC82F82E090E090
:10029000C53028F40AD003DFEACFC81BF7CFEADE67
:1002A00081E090E0F7CFF7DEE2CFE199FECF8EBBA1
:1002B000E09A99278DB30895262FE199FECF1CBAB5
:1002C0008EBB2DBB0FB6F894E29AE19A0FBE019651
:0602D0000895F894FFCF31
:00000001FF
